:020000020000FC
:1000000009C007C006C005C004C003C002C001C0CB
:1000100000C0189500E801BFC09A01E007BB00E7E7
:1000200005BF1BE53FD01FEF48D01FEF46D01FEFA5
:1000300044D01FEF42D01AE540D01BE133D019E382
:100040003CD018E12FD019E838D01BE12BD01FEF9E
:1000500034D01FEF32D01FEF30D01FEF2ED01FEF64
:100060002CD01FEF2AD01FEF28D01FEF26D01FEF74
:1000700024D01FEF22D01BE515D01FEF1ED01FEF9D
:100080001CD01FEF1AD01FEF18D01AE516D01BE1B5
:1000900009D019E312D018E105D019E80ED01BE100
:1000A00001D0889503E0C0980A95E9F703E0C09A6B
:1000B0000A95E9F71A95B1F7089503E0C09A0A95F1
:1000C000E9F703E0C09A0A95E9F71A95B1F70895A0
:00000001FF
